:020000040000FA
:0400000081EF00F09C
:100008008E408E408E408E404000484040008E40DA
:100018008C408E408E408E408E408E408E408E406A
:100028008E404000400040008E408E408E408E4002
:100038008E408E408E408E408E408E408E408E4048
:100048008E408E408E408E40400040008E408E4054
:100058008E408E408E4040008E408E408E408E40B6
:100068008E408E408E408E408E408E408E408E4018
:100078008E408E408E408E4040008E408E408E4096
:100088008E408E408E408E408E408E408E408E40F8
:100098008E408E408E408E4040008E404000400092
:1000A8008E408E408E408E408E408E408E408E40D8
:1000B8008E408E408E408E408E408E408E408E40C8
:1000C8008E408E408E408E408E408E408E408E40B8
:1000D8008E408E408E408E408E408E408E408E40A8
:1000E80040008E408E408E4040004000400040005E
:0E00F8008E408E408E408E40FF0000EF81F063
:10DFFE0000F331ED80C34100FFC33400FFFFFFFF8C
:10E00E00FFC31B00FFFFFFFFFFC32E003A01E0CB53
:10E01E004728F93A00E0FE61D8FE7BD0E6DFC93A28
:10E02E0001E0CB47C9F53A01E0CB4F28F9F13200B8
:10E03E00E0C9C34400C34A00C3BF00C35100020974
:10E04E007810214580F9C3931C11290306632145DD
:10E05E00801A77231305C26000F9CD2A05CDF80A80
:10E06E0032EF80323E8121A281237CB5CA87007EA9
:10E07E00472F77BE70CA78002B11A181CDC006DA6A
:10E08E00C80011CEFF22F48019229F80CD05052AEB
:10E09E009F8011EFFF19113E817D936F7C9A67E58A
:10E0AE0021E000CD9611E1CD391821D100CD961188
:10E0BE0031AB80CD2A05C34304211701CD9611C380
:10E0CE00CE0020427974657320667265650D0A0074
:10E0DE00005A38302042415349432056657220344D
:10E0EE002E37620D0A436F70797269676874202843
:10E0FE0043292031393738206279204D6963726F98
:10E10E00736F66740D0A00004D656D6F7279207322
:10E11E00697A65206E6F7420656E6F7567680D0A7B
:10E12E005468652073797374656D206973207374F8
:10E13E006F707065642E0D0A0000AE167217C4164D
:10E14E0048805610DB1384103819171A5315861988
:10E15E008C1A921AF31A081B2F14731B968008132D
:10E16E002011A21317132813951B281C381368139C
:10E17E007213C54E44C64F52CE455854C4415441F5
:10E18E00C94E505554C4494DD2454144CC4554C74F
:10E19E004F544FD2554EC946D24553544F5245C790
:10E1AE004F535542D2455455524ED2454DD3544FEE
:10E1BE0050CF5554CF4ECE554C4CD7414954C445F3
:10E1CE0046D04F4B45C44F4B45D3435245454ECC9D
:10E1DE00494E4553C34C53D749445448CD4F4E49ED
:10E1EE00544F52D34554D245534554D052494E54B0
:10E1FE00C34F4E54CC495354C34C454152C34C4F5C
:10E20E004144C353415645CE4557D4414228D44F7D
:10E21E00C64ED3504328D448454ECE4F54D35445C2
:10E22E0050ABADAAAFDEC14E44CF52BEBDBCD3473C
:10E23E004EC94E54C14253D55352C65245C94E5083
:10E24E00D04F53D35152D24E44CC4F47C55850C3E2
:10E25E004F53D3494ED4414EC1544ED045454BC475
:10E26E0045454BD04F494E54CC454ED3545224D6EF
:10E27E00414CC15343C3485224C8455824C2494E49
:10E28E0024CC45465424D24947485424CD494424ED
:10E29E00809A089707720CE709790BAE0EA80BFE51
:10E2AE0009A4098709760A60089309C209E9099841
:10E2BE0008E713580AD908ED138C1036147E1BE9A3
:10E2CE0009641B571B5C1B901C99809C809A0AC684
:10E2DE00080C074109E909E9090405792018795460
:10E2EE00147C92157CF3157F411950070E46060ECD
:10E2FE004E46534E52474F4446434F564F4D554C44
:10E30E00425344442F304944544D4F534C5353546D
:10E31E00434E55464D4F4858424EC3BF00C3170992
:10E32E00D300C9D6006F7CDE006778DE00473E0062
:10E33E00C9000000354ACA99391C76982295B398BF
:10E34E000ADD479853D199990A1A9F9865BCCD98C2
:10E35E00D6773E9852C74F80DB00C901FF1C0000E4
:10E36E001400140000000000C33D06C30000C300EB
:10E37E0000C30000A281FEFF3F81204572726F72C2
:10E38E000020696E20004F6B0D0A0000427265611D
:10E39E006B00210400397E23FE81C04E234623E507
:10E3AE0069607AB3EBCABB03EBCDC006010D00E189
:10E3BE00C809C3A503CDDE03C5E3C1CDC0067E02E9
:10E3CE00C80B2BC3CA03E52A1F81060009093EE5C7
:10E3DE003ED0956F3EFF9CDAED036739E1D81E0CF7
:10E3EE00C30C042A0E8122A1801E02011E14011EDE
:10E3FE0000011E12011E22011E0A011E18CD2A0541
:10E40E00328A80CDEB0A21FF02573E3FCDD106194D
:10E41E007ECDD106CD5008CDD106218903CD9611E2
:10E42E002AA18011FEFFCDC006CA51007CA53CC4B6
:10E43E0031183EC1AF328A80CDEB0A219503CD96BD
:10E44E001121FFFF22A180CD3D06DA5004CD5008E8
:10E45E003C3DCA5004F5CD1C09D5CD540547D1F12C
:10E46E00D23008D5C5AF321181CD5008B7F5CDE405
:10E47E0004DA8904F1F5CABD09B7C5D2A004EB2AA6
:10E48E001B811A020313CDC006C291046069221BC0
:10E49E0081D1F1CAC7042A1B81E3C109E5CDC403AA
:10E4AE00E1221B81EB74D123237323722311A680E7
:10E4BE001A772313B7C2BF04CD100523EB626B7E10
:10E4CE0023B6CA5004232323AFBE23C2D804EB7352
:10E4DE002372C3CC042AA380444D7E23B62BC823BB
:10E4EE00237E23666FCDC00660697E23666F3FC8AC
:10E4FE003FD0C3E704C02AA380AF77237723221B24
:10E50E00812AA3802B2213812AF480220881AFCD89
:10E51E0060082A1B81221D81221F81C12A9F80F93A
:10E52E0021F88022F680AF6F672219813210812286
:10E53E002381E5C52A1381C93E3FCDD1063E20CDAC
:10E54E00D106C39380AF32F3800E0511A6807EFEF6
:10E55E0020CADC0547FE22CAFC05B7CA03063AF3F9
:10E56E0080B77EC2DC05FE3F3E9ECADC057EFE30D5
:10E57E00DA8705FE3CDADC05D5118001C501D80528
:10E58E00C5067F7EFE61DAA005FE7BD2A005E65FA2
:10E59E00774EEB23B6F2A205047EE67FC8B9C2A27F
:10E5AE0005EBE5131AB7FAD4054F78FE88C2C305FA
:10E5BE00CD50082B237EFE61DACC05E65FB9CAB2D8
:10E5CE0005E1C3A00548F1EBC9EB79C1D1231213C4
:10E5DE000CD63ACAEA05FE49C2ED0532F380D6548E
:10E5EE00C25D05477EB7CA0306B8CADC0523120C06
:10E5FE0013C3F30521A5801213121312C93A898091
:10E60E00B73E00328980C2200605CA3D06CDD1062E
:10E61E003E052BCA34067ECDD106C34606052BCD4C
:10E62E00D106C24606CDD106CDF80AC33D0621A6B7
:10E63E00800601AF328980CDFB064FFE7FCA0C06E5
:10E64E003A8980B7CA5F063E00CDD106AF328980C7
:10E65E0079FE07CAA306FE03CCF80A37C8FE0DCA18
:10E66E00F30AFE15CA3706FE40CA3406FE5FCA2CF0
:10E67E0006FE08CA2C06FE12C29E06C5D5E5360059
:10E68E00CDA21C21A680CD9611E1D1C1C34606FEB6
:10E69E0020DA460678FE493E07D2B8067971321165
:10E6AE00812304CDD106C34606CDD1063E08C3B2A2
:10E6BE00067C92C07D93C97EE3BE23E3CA5008C395
:10E6CE00F803F53A8A80B7C2CB11F1C5F5FE20DA10
:10E6DE00F5063A8780473AF08004CAF10605B8CCB1
:10E6EE00F80A3C32F080F1C1CD8D1CC9CD551BE628
:10E6FE007FFE0FC03A8A802F328A80AFC9CD1C09A7
:10E70E00C0C1CDE404C5CD6207E14E23462378B1E6
:10E71E00CA4304CD6B07CD7B08C5CDF80A5E2356E0
:10E72E0023E5EBCD39183E20E1CDD1067EB723CAC5
:10E73E001807F23807D67F4F1181011A13B7F24A24
:10E74E00070DC24A07E67FCDD1061A13B7F254075A
:10E75E00C33B07E52A8D80228B80E1C9E5D52A8B44
:10E76E008011FFFFED5A228B80D1E1F0E52A8D80DA
:10E77E00228B80CD551BFE03CA8E07E1C36B072A81
:10E78E008D80228B80C3C2003E64321081CDFE0983
:10E79E00C1E5CDE709220C8121020039CDA503D1B7
:10E7AE00C2C70709D52B562B5E2323E52A0C81CD34
:10E7BE00C006E1C2AB07D1F9EB0E08CDD503E52AB1
:10E7CE000C81E3E52AA180E3CDC00CCDC606A6CD13
:10E7DE00BD0CE5CDEB16E1C5D5010081515A7EFE8B
:10E7EE00AB3E01C20308CD5008CDBD0CE5CDEB16F6
:10E7FE00CD9F16E1C5D5F533E52A1381E30681C514
:10E80E0033CD7B082213817EFE3ACA3008B7C2F898
:10E81E0003237E23B6CAA208235E2356EB22A180D1
:10E82E00EBCD5008111008D5C8D680DAFE09FE25AA
:10E83E00D2F803074F0600EB21A002094E2346C56E
:10E84E00EB237EFE3AD0FE20CA5008FE303F3C3D00
:10E85E00C9EB2AA380CA7508EBCD1C09E5CDE404EB
:10E86E006069D1D2BD092B222181EBC9DFC8D7FE49
:10E87E001B2811FE03280DFE13C0D7FE11C8FE0380
:10E88E00280718F63EFF329280C0F6C0221381216F
:10E89E00F6FFC12AA180F57DA43CCAB508221781D6
:10E8AE002A1381221981AF328A80CDEB0AF1219B86
:10E8BE0003C22C04C343042A19817CB51E20CA0C42
:10E8CE0004EB2A178122A180EBC9CD1E14C032861B
:10E8DE0080C9E52A8F8006004F09228F80E1C97E0C
:10E8EE00FE41D8FE5B3FC9CD5008CDBD0CCD9F1665
:10E8FE00FA17093A2C81FE90DA4717018090110021
:10E90E0000E5CD1A17E151C81E08C30C042B1100E7
:10E91E0000CD5008D0E5F5219819CDC006DAF803E0
:10E92E00626B19291929F1D6305F160019EBE1C374
:10E93E002009CA1405CDF9082BCD5008E52AF4801C
:10E94E00CA6409E1CDC6062CD5CDF9082BCD5008E9
:10E95E00C2F803E3EB7D935F7C9A57DAED03E52A69
:10E96E001B8101280009CDC006D2ED03EB229F804A
:10E97E00E122F480E1C31405CA1005CD140501107F
:10E98E0008C3A3090E03CDD503C1E5E52AA180E393
:10E99E003E8CF533C5CD1C09CDE909E52AA180CD04
:10E9AE00C006E123DCE704D4E40460692BD81E0E14
:10E9BE00C30C04C016FFCDA103F9FE8C1E04C20CBD
:10E9CE0004E122A180237CB5C2E1093A1181B7C2CC
:10E9DE004204211008E33EE1013A0E000600794898
:10E9EE00477EB7C8B8C823FE22CAED09C3F009CDC9
:10E9FE00B30ECDC606B4D53AF280F5CDCF0CF1E309
:10EA0E002213811FCDC20CCA510AE52A2981E523A2
:10EA1E00235E23562AA380CDC006D2400A2A9F80A9
:10EA2E00CDC006D1D2480A210481CDC006D2480AF3
:10EA3E003ED1CDF712EBCD3011CDF712E1CDFA1656
:10EA4E00E1C9E5CDF716D1E1C9CD1E147E47FE8C86
:10EA5E00CA670ACDC606882B4B0D78CA3808CD1D5D
:10EA6E0009FE2CC0C3680ACDCF0C7EFE88CA840A6C
:10EA7E00CDC606A92BCDC00CCD9F16CAE909CD5027
:10EA8E0008DAA409C337082BCD5008CAF80AC8FE05
:10EA9E00A5CA2B0BFEA8CA2B0BE5FE2CCA140BFE27
:10EAAE003BCA4E0BC1CDCF0CE53AF280B7C2E40A99
:10EABE00CD4418CD541136202A2981342A29813A81
:10EACE0087804704CAE00A043AF080863DB8D4F83D
:10EADE000ACD9911AFC49911E1C3960A3AF080B7E5
:10EAEE00C8C3F80A360021A5803E0DCDD1063E0AD8
:10EAFE00CDD106AF32F0803A86803DC8F5AFCDD18C
:10EB0E0006F1C3090B3A8880473AF080B8D4F80A68
:10EB1E00D24E0BD60ED2220B2FC3430BF5CD1B14A8
:10EB2E00CDC606292BF1D6A8E5CA3E0B3AF0802FAA
:10EB3E0083D24E0B3C473E20CDD10605C2470BE19A
:10EB4E00CD5008C39D0A3F5265646F2066726F6D8B
:10EB5E002073746172740D0A003A1281B7C2F20307
:10EB6E00C121550BCD9611C34305CD01117EFE2259
:10EB7E003E00328A80C2930BCD5511CDC6063BE5C1
:10EB8E00CD99113EE5CD4705C1DA9F08237EB72BFF
:10EB9E00C5CAE609362CC3AD0BE52A2181F6AF3284
:10EBAE001281E3C3B90BCDC6062CCDB30EE3D57ED1
:10EBBE00FE2CCAE10B3A1281B7C24E0C3E3FCDD1AC
:10EBCE0006CD4705D1C1DA9F08237EB72BC5CAE60D
:10EBDE0009D53AF280B7CA0B0CCD50085747FE2222
:10EBEE00CAFF0B3A1281B757CAFC0B163A062C2BEA
:10EBFE00CD5811EB21160CE3D5C3190ACD5008CD13
:10EC0E00A617E3CDF716E12BCD5008CA220CFE2C29
:10EC1E00C2680BE32BCD5008C2B50BD13A1281B7A7
:10EC2E00EBC27608D5B6213D0CC49611E1C93F451D
:10EC3E00787472612069676E6F7265640D0A00CD1B
:10EC4E00E709B7C2670C237E23B61E06CA0C04233F
:10EC5E005E2356EB220E81EBCD5008FE83C24E0C86
:10EC6E00C3E10B110000C4B30E221381CDA103C268
:10EC7E00FE03F9D57E23F5D5CDDD16E3E5CD4A1499
:10EC8E00E1CDF716E1CDEE16E5CD1A17E1C190CD27
:10EC9E00EE16CAAD0CEB22A1806960C30C08F92AEE
:10ECAE0013817EFE2CC21008CD5008CD750CCDCF31
:10ECBE000CF6373AF2808FB7E8C30A04CDC60628A1
:10ECCE002B1600D50E01CDD503CD460D2215812A6A
:10ECDE001581C178FE78D4C00C7E1600D6B3DA0743
:10ECEE000DFE03D2070DFE0117AABA57DAF803225A
:10ECFE000A81CD5008C3EB0C7AB7C22E0E7E220AC3
:10ED0E0081D6ACD8FE07D05F3AF2803DB37BCA8C79
:10ED1E001207835F21EA02197856BAD023CDC00CB0
:10ED2E00C501DE0CC5434ACDD01658514E2346239D
:10ED3E00C52A0A81C3D20CAF32F280CD50081E24F0
:10ED4E00CA0C04DAA617CDEE08D2AD0DFE2620129F
:10ED5E00CD5008FE48CAEA1BFE42CA5A1C1E02CA01
:10ED6E000C04FEACCA460DFE2ECAA617FEADCA9CFA
:10ED7E000DFE22CA5511FEAACA8E0EFEA7CAB910E2
:10ED8E00D6B6D2BE0DCDCB0CCDC60629C9167DCDBD
:10ED9E00D20C2A1581E5CDC816CDC00CE1C9CDB374
:10EDAE000EE5EB2229813AF280B7CCDD16E1C906D9
:10EDBE0000074FC5CD500879FE31DAE50DCDCB0CED
:10EDCE00CDC6062CCDC10CEB2A2981E3E5EBCD1E79
:10EDDE0014EBE3C3ED0DCD940DE311A80DD5014950
:10EDEE0001094E236669E915FEADC8FE2DC814FE55
:10EDFE002BC8FEACC82BC9F6AFF5CDC00CCD0209A1
:10EE0E00F1EBC1E3EBCDE016F5CD0209F1C17921AD
:10EE1E007710C2290EA34F78A2E9B34F78B2E92139
:10EE2E00400E3AF2801F7A175F166478BAD0C32F5D
:10EE3E000D420E79B71FC1D1F5CDC20C21840EE55E
:10EE4E00CA1A17AF32F280D5CDD9127E23234E23A4
:10EE5E0046D1C5F5CDDD12CDEE16F157E17BB2C828
:10EE6E007AD601D8AFBB3CD0151D0ABE2303CA6C9F
:10EE7E000E3FC3AA163C8FC1A0C6FF9FC3B1161684
:10EE8E005ACDD20CCDC00CCD02097B2F4F7A2FCD8F
:10EE9E007710C1C3DE0C2BCD5008C8CDC6062C0191
:10EEAE00A50EC5F6AF32F18046CDEE08DAF803AF07
:10EEBE004F32F280CD5008DACF0ECDEE08DADC0EEE
:10EECE004FCD5008DAD00ECDEE08D2D00ED624C2D9
:10EEDE00EB0E3C32F2800F814FCD50083A10813D3F
:10EEEE00CA980FF2FB0E7ED628CA700FAF32108171
:10EEFE00E550592A2381CDC006112581CAE0152A75
:10EF0E001D81EB2A1B81CDC006CA2E0F799623C216
:10EF1E00230F789623CA620F23232323C3150FE1F1
:10EF2E00E3D511B00DCDC006D1CA650FE3E5C5011D
:10EF3E0006002A1F81E509C1E5CDC403E1221F8128
:10EF4E006069221D812B3600CDC006C2540FD173CD
:10EF5E00237223EBE1C9322C81219403222981E112
:10EF6E00C9E52AF180E357D5C5CDF608C1F1EBE32B
:10EF7E00E5EB3C577EFE2CCA760FCDC60629221530
:10EF8E0081E122F1801E00D511E5F52A1D813E1981
:10EF9E00EB2A1F81EBCDC006CAD00F7EB923C2B2B9
:10EFAE000F7EB8235E235623C29E0F3AF180B7C25E
:10EFBE000104F1444DCAE01596CA2E101E10C30C62
:10EFCE0004110400F1CA1709712370234FCDD50324
:10EFDE002323220A8171233AF1801779010B00D283
:10EFEE00F30FC10371237023F5E5CD8B17EBE1F120
:10EFFE003DC2EB0FF5424BEB19DAED03CDDE0322EA
:10F00E001F812B3600CDC006C2111003572A0A816C
:10F01E005EEB2909EB2B2B73237223F1DA52104787
:10F02E004F7E2316E15E235623E3F5CDC006D2CBE9
:10F03E000FE5CD8B17D119F13D444DC2331029295F
:10F04E00C109EB2A1581C92A1F81EB210000393A2B
:10F05E00F280B7CA7210CDD912CDD9112A9F80EB8A
:10F06E002A08817D934F7C9A41501E0021F28073B5
:10F07E000690C3B6163AF08047AFC37810CD0F1185
:10F08E00CD011101E709C5D5CDC60628CDB30EE5D4
:10F09E00EB2B562B5EE1CDC00CCDC60629CDC60698
:10F0AE00B4444DE3712370C34E11CD0F11D5CD94E1
:10F0BE000DCDC00CE35E2356237AB3CA04047E231F
:10F0CE00666FE52A2381E32223812A2781E52A25FB
:10F0DE0081E5212581D5CDF716E1CDBD0C2BCD5087
:10F0EE0008C2F803E1222581E1222781E122238152
:10F0FE00E1C9E52AA180237CB5E1C01E16C30C042C
:10F10E00CDC606A73E80321081B647CDB80EC3C01D
:10F11E000CCDC00CCD4418CD5411CDD912013413E1
:10F12E00C57E2323E5CDAF11E14E2346CD4811E533
:10F13E006FCDCC12D1C9CDAF11210481E577232338
:10F14E00732372E1C92B062250E50EFF237E0CB706
:10F15E00CA6A11BACA6A11B8C25B11FE22CC500833
:10F16E00E323EB79CD48111104812AF680222981FF
:10F17E003E0132F280CDFA16CDC00622F680E17E37
:10F18E00C01E1EC30C0423CD5411CDD912CDEE16C4
:10F19E001C1DC80ACDD106FE0DCC020B03C3A01157
:10F1AE00B70EF1F52A9F80EB2A08812F4F06FF0933
:10F1BE0023CDC006DACD1122088123EBF1C9F11E51
:10F1CE001ACA0C04BFF501B111C52AF480220881B8
:10F1DE00210000E52A9F80E521F880EB2AF680EBDE
:10F1EE00CDC00601EA11C23E122A1B81EB2A1D81F7
:10F1FE00EBCDC006CA11127E2323B7CD4112C3FB3D
:10F20E0011C1EB2A1F81EBCDC006CA6712CDEE16D7
:10F21E007BE509B7F21012220A81E14E06000909B8
:10F22E0023EB2A0A81EBCDC006CA1112013012C59A
:10F23E00F6807E23235E235623F0B7C8444D2A085A
:10F24E0081CDC0066069D8E1E3CDC006E3E5606913
:10F25E00D0C1F1F1E5D5C5C9D1E17DB4C82B462B9E
:10F26E004EE52B2B6E26000950592B444D2A088152
:10F27E00CDC703E171237069602BC3DC11C5E52A8C
:10F28E002981E3CD460DE3CDC10C7EE52A2981E52A
:10F29E00861E1CDA0C04CD4511D1CDDD12E3CDDC7A
:10F2AE0012E52A0681EBCDC312CDC31221DB0CE38E
:10F2BE00E5C37611E1E37E23234E23466F2C2DC842
:10F2CE000A120313C3CD12CDC10C2A2981EBCDF73F
:10F2DE0012EBC0D550591B4E2A0881CDC006C2F57F
:10F2EE00124709220881E1C92AF6802B462B4E2BA4
:10F2FE002BCDC006C022F680C9018710C5CDD6120F
:10F30E00AF5732F2807EB7C9018710C5CD0C13CA34
:10F31E00170923235E23561AC93E01CD4511CD216F
:10F32E00142A068173C1C37611CDD113AFE34FE515
:10F33E007EB8DA461378110E00C5CDAF11C1E1E5E6
:10F34E00232346236668060009444DCD48116FCD30
:10F35E00CC12D1CDDD12C37611CDD113D1D51A90E9
:10F36E00C33C13EB7ECDD6130405CA1709C51EFF89
:10F37E00FE29CA8B13CDC6062CCD1E14CDC606296A
:10F38E00F1E3013E13C53DBE0600D04F7E91BB4753
:10F39E00D843C9CD0C13CABF145F23237E23666FD7
:10F3AE00E5194672E3C57EFE24C2C013CDEA1B18D2
:10F3BE000DFE25C2CA13CD5A1C1803CDA617C1E1E6
:10F3CE0070C9EBCDC60629C1D1C543C9CD211432B2
:10F3DE008480CD8380C38710CD0B14C34B80CD0B9F
:10F3EE0014F51E002BCD5008CA0114CDC6062CCD27
:10F3FE001E14C1CD8380ABA0CA0214C9CD1E143217
:10F40E008480324C80CDC6062CC31E14CD5008CD40
:10F41E00BD0CCDFC087AB7C217092BCD50087BC99D
:10F42E00CD02091AC38710CDBD0CCD0209D5CDC6AC
:10F43E00062CCD1E14D112C9211D19CDEE16C3599D
:10F44E0014CDEE1621C1D1CDC81678B7C83A2C818D
:10F45E00B7CAE01690D273142F3CEBCDD016EBCD7D
:10F46E00E016C1D1FE19D0F5CD051767F1CD1E15E9
:10F47E00B4212981F29914CDFE14D2DF142334CA9B
:10F48E0007042E01CD3415C3DF14AF90477E9B5F6A
:10F49E00237E9A57237E994FDC0A156863AF47790E
:10F4AE00B7C2CC144A54656F78D608FEE0C2AD14CC
:10F4BE00AF322C81C905297A1757798F4FF2C414B0
:10F4CE00785C45B7CADF14212C818677D2BF14C869
:10F4DE0078212C81B7FCF11446237EE680A94FC318
:10F4EE00E0161CC014C00CC00E8034C0C307047ECE
:10F4FE00835F237E8A57237E894FC9212D817E2FDC
:10F50E0077AF6F90477D9B5F7D9A577D994FC90668
:10F51E0000D608DA2D15435A510E00C32015C60920
:10F52E006FAF2DC8791F4F7A1F577B1F5F781F470C
:10F53E00C330150000008103AA561980F12276808F
:10F54E0045AA3882CD9F16B7EA1709212C817E0174
:10F55E00358011F30490F570D5C5CD5914C1D10481
:10F56E00CDF515214215CD5014214615CDE71901C3
:10F57E008080110000CD5914F1CD1A18013180117F
:10F58E00187221C1D1CD9F16C82E00CD5D167932CD
:10F59E003B81EB223C81010000505821AA14E52149
:10F5AE00B615E5E52129817E23B7CAE215E52E08B9
:10F5BE001F6779D2D015E52A3C8119EBE13A3B81E0
:10F5CE00891F4F7A1F577B1F5F781F472D7CC2BF45
:10F5DE0015E1C9435A514FC9CDD0160120841100EF
:10F5EE0000CDE016C1D1CD9F16CAFB032EFFCD5D17
:10F5FE001634342B7E3257802B7E3253802B7E3244
:10F60E004F8041EBAF4F575F325A80E5C57DCD4EEF
:10F61E0080DE003FD22D16325A80F1F137D2C1E191
:10F62E00793C3D1FFAE014177B175F7A175779174D
:10F63E004F297817473A5A8017325A8079B2B3C297
:10F64E001A16E5212C8135E1C21A16C3070478B7C4
:10F65E00CA81167D212C81AE80471FA878F28016B4
:10F66E00C68077CAE015CD0517772BC9CD9F162F0B
:10F67E00E1B7E1F2BF14C30704CDEB1678B7C8C6E5
:10F68E0002DA070447CD5914212C8134C0C3070474
:10F69E003A2C81B7C83A2B81FE2F179FC03CC9CD9B
:10F6AE009F160688110000212C814F70060023360C
:10F6BE008017C3A714CD9F16F0212B817EEE807785
:10F6CE00C9EB2A2981E3E52A2B81E3E5EBC9CDEECF
:10F6DE0016EB2229816069222B81EBC92129815EDB
:10F6EE002356234E234623C911298106041A771364
:10F6FE002305C2FC16C9212B817E07371F773F1FBA
:10F70E002323777907371F4F1FAEC978B7CA9F16C5
:10F71E0021A816E5CD9F1679C8212B81AE79F8CD9B
:10F72E0034171FA9C92378BEC02B79BEC02B7ABE51
:10F73E00C02B7B96C0E1E1C9474F575FB7C8E5CDF7
:10F74E00EB16CD0517AE67FC6B173E9890CD1E15C8
:10F75E007C17DCF1140600DC0A15E1C91B7AA33C08
:10F76E00C00BC9212C817EFE983A2981D07ECD47CF
:10F77E001736987BF57917CDA714F1C921000078BB
:10F78E00B1C83E1029DACB0FEB29EBD2A11709DA5B
:10F79E00CB0F3DC29317C9FE2DF5CAB217FE2BCA69
:10F7AE00B2172BCDBF1447575F2F4FCD5008DA033A
:10F7BE0018FE2ECADE17FE45C2E217CD5008CDF652
:10F7CE000DCD5008DA251814C2E217AF935F0C0C5A
:10F7DE00CABA17E57B90F4FB17F2F117F5CDE715D2
:10F7EE00F13CC2E517D1F1CCC816EBC9C8F5CD88EE
:10F7FE0016F13DC9D557788947C5E5D5CD8816F19F
:10F80E00D630CD1A18E1C1D1C3BA17CDD016CDB1AD
:10F81E0016C1D1C359147B0707830786D6305FC341
:10F82E00D017E5219003CD9611E1EBAF0698CDB63A
:10F83E0016219511E5212E81E5CD9F163620F25227
:10F84E0018362D233630CA0819E5FCC816AFF5CD8B
:10F85E000E1901439111F84FCD1A17B7E27F18F127
:10F86E00CDFC17F5C36118CDE715F13CF5CD0E199A
:10F87E00CD47143CCD4717CDE016010603F1813C70
:10F88E00FA9B18FE08D29B183C473E023D3DE1F51F
:10F89E0011211905C2AC18362E2336302305362E0B
:10F8AE00CCF516C5E5D5CDEB16E1062F047B965F9C
:10F8BE00237A9E5723799E4F2B2BD2BB18CDFE1445
:10F8CE0023CDE016EBE17023C10DC2AC1805CAECD6
:10F8DE00182B7EFE30CAE018FE2EC4F516F1CA0BA8
:10F8EE0019364523362BF2FC18362D2F3C062F04E5
:10F8FE00D60AD2FE18C63A237023772371E1C901C6
:10F90E00749411F723CD1A17B7E1E27618E90000C7
:10F91E000080A08601102700E803006400000A00A2
:10F92E000001000021C816E3E9CDD016211D19CD26
:10F93E00DD16C1D1CD9F1678CA8619F25119B7CAF4
:10F94E00FB03B7CAC014D5C579F67FCDEB16F26EA0
:10F95E0019D5C5CD7217C1D1F5CD1A17E17C1FE1AE
:10F96E00222B81E1222981DC3319CCC816D5C5CDD5
:10F97E005315C1D1CD9415CDD016013881113BAAA6
:10F98E00CD94153A2C81FE88D27B16CD7217C68087
:10F99E00C602DA7B16F5214215CD4A14CD8B15F130
:10F9AE00C1D1F5CD5614CDC81621C619CDF61911F3
:10F9BE000000C14AC3941508402E9474704F2E77E0
:10F9CE006E02887AE6A02A7C50AAAA7EFFFF7F7F6D
:10F9DE000000808100000081CDD016119215D5E572
:10F9EE00CDEB16CD9415E1CDD0167E23CDDD1606CA
:10F9FE00F1C1D13DC8D5C5F5E5CD9415E1CDEE16D5
:10FA0E00E5CD5914E1C3FF19CD9F16215E80FA781A
:10FA1E001A217F80CDDD16215E80C886E60706009E
:10FA2E00772387874F09CDEE16CD94153A5D803C2E
:10FA3E00E6030600FE0188325D80217C1A87874F1F
:10FA4E0009CD4A14CDEB167B59EE4F4F36802B461F
:10FA5E003680215C80347ED6ABC26F1A770C151CB3
:10FA6E00CDAA14217F80C3F716772B772B77C3533C
:10FA7E001A68B1466899E9926910D1756821D61A4B
:10FA8E00CD4A14CDD01601498311DB0FCDE016C13E
:10FA9E00D1CDF515CDD016CD7217C1D1CD561421BD
:10FAAE00DA1ACD5014CD9F1637F2C21ACD4714CDA7
:10FABE009F16B7F5F4C81621DA1ACD4A14F1D4C838
:10FACE001621DE1AC3E719DB0F49810000007F05FE
:10FADE00BAD71E866426998758342387E05DA5869B
:10FAEE00DA0F4983CDD016CD921AC1E1CDD016EBE7
:10FAFE00CDE016CD8C1AC3F315CD9F16FC3319FC31
:10FB0E00C8163A2C81FE81DA251B0100815159CD90
:10FB1E00F515215014E5212F1BCDE71921D61AC951
:10FB2E00094AD73B78026E847BFEC12F7C74319AD2
:10FB3E007D843D5A7DC87F917EE4BB4C7E6CAAAA23
:10FB4E007F00000081C9D7C93E0CC38D1CCD1E1489
:10FB5E007B328780C9CDBD0CCD0209ED538B80ED74
:10FB6E00538D80C9CD0209D5E146237EC37810CDD1
:10FB7E00BD0CCD0209D5CDC6062CCDBD0CCD0209CE
:10FB8E00E3732372E1C9CDC00CCD0209C5212E81CC
:10FB9E007AFE00280CCDCD1B78FE30280270237122
:10FBAE00237BCDCD1B7AFE00200578FE3028027017
:10FBBE00237123AF772377C1212E81C3261147E608
:10FBCE000FFE0A3802C607C6304F780F0F0F0FE62A
:10FBDE000FFE0A3802C607C63047C9EB210000CD1A
:10FBEE00031CDA231C1805CD031C381F29292929CB
:10FBFE00B56F18F3131AFE20CA031CD630D8FE0AAE
:10FC0E003805D607FE0AD8FE103FC9EB7A4BE5CD74
:10FC1E007710E1C91E26C30C04CDC00CCD0209C558
:10FC2E00212E8106110578FE012808CB13CB123048
:10FC3E00F41804CB13CB123E30CE0077230520F3FD
:10FC4E00AF772377C1212E81C32611EB210000CD82
:10FC5E00771CDA851CD63029B56FCD771C30F6EBC4
:10FC6E007A4BE5CD7710E1C9131AFE20CA771CFE38
:10FC7E0030D8FE323FC91E28C30C04C35100C3083E
:10FC8E0000C300003E00329280C35800F5A0C1B8F8
:10FC9E003E00C9CDD106C3F80AFFFFFFFFFFFFFFED
:10FCAE00FFFFFFFFFFFFFFFFFFFFFFFFFFFFFFFF56
:10FCBE00FFFFFFFFFFFFFFFFFFFFFFFFFFFFFFFF46
:10FCCE00FFFFFFFFFFFFFFFFFFFFFFFFFFFFFFFF36
:10FCDE00FFFFFFFFFFFFFFFFFFFFFFFFFFFFFFFF26
:02FFFE00FF0002
:020000040001F9
:10000000080E0001B16F000E0401186F1969C9686C
:10001000000E086F0969C768000E106F1169C86883
:1000200020912181CA802093C292CA922095C284D5
:10003000CA9400910181C680009B018BC68A3F0E45
:100040000201046F04010097C696010E456F400E31
:10005000446F2F0E436F000E476F4691468B468FBD
:10006000010E0201D56FA00ED46FD189D18B04018E
:10007000009FC68E070E0201766F0401009DBE8CA4
:10008000C69C260E0201076FD28F040100930183E4
:10009000C682010E0201616F040100950185C684CC
:1000A000020E0201626F04010099BE88C698010E1B
:1000B0000201056F000E0001D56F820ED76F000E92
:1000C000D86F010ED96F7F0EDA6F7F0EDB6F010ED6
:1000D000DC6F040EDD6F000EDE6F000EDF6F000EB2
:1000E000D46F8C0ED66FD68A550E0401596FAA0EA6
:1000F000596F5991000E5F6F000E5E6F080E5D6FB5
:10010000550E596FAA0E596F5981AE9A9E8A010EEB
:0E01100002013E6FD6809F80D68EC282FFD73E
:100120006100D8F301F56100DCF302F56100E0F352
:1001300003F56100D4F304F5AE9A610044F306F5CB
:1001400061003CF305F5CEBA34D0000EC86E200E27
:10015000065CD8B00AD0FF0E0524F66EDF0E06202E
:10016000F76E0800F5C4C0F43BD0800E065CD8A042
:100170000DD0900E065CD8B009D0000E0524D96EC3
:10018000960E0620DA6EDF50C06E2AD0050407E115
:10019000E00E0618D8A403D0B7C4C0F421D0E00EF6
:1001A00006180510D8A403D0C7C2C0F419D0C0687F
:1001B00017D0800E065CD8A00DD0900E065CD8B08B
:1001C00009D0000E0524D96E960E0620DA6ED0C432
:1001D000DFF406D0E00E06180510D8B4D0C4C9F27A
:1001E0000001D785D795610010F4F5F461000CF497
:1001F000F8F4610008F4F7F4610004F4F6F4110077
:1002000005EE00F214EE00F0EE6AE550E150FCE17C
:10021000E250FAE1066A056A0401080E5D6F000EFD
:100220005E6F000E5F6F000EF86E000100EF80F051
:06023000AF90C868110048
:020238001100B3
:020000040020DA
:10000000FF0FFF0FFF0FFF0FFF0FFF0FFF0FFF0F80
:10001000FF0FFF0FFF0FFF0FFF0FFF0FFF0FFF0F70
:020000040030CA
:0A0000008CFFFFF79FFFFFFFFFFFDB
:00000001FF
